:020000040000fa
:04005c00fa020000a4
:020000040000fa
:04000c00fa020000f4
:020000040000fa
:04007000fa02000090
:020000040000fa
:04007400fa0200008c
:020000040000fa
:04013400fa020000cb
:020000040000fa
:04015c00fa020000a3
:020000040000fa
:04003800fa020000c8
:020000040000fa
:04006000fa020000a0
:020000040000fa
:04008800fa02000078
:020000040000fa
:0400b800fa02000048
:020000040000fa
:04001c00fa020000e4
:020000040000fa
:04001000fa020000f0
:020000040000fa
:04002c00fa020000d4
:020000040000fa
:04003c00fa020000c4
:020000040000fa
:0400bc00fa02000044
:020000040000fa
:0400c000fa02000040
:020000040000fa
:04026000fa0200009e
:020000040000fa
:04002800fa020000d8
:020000040000fa
:04007800fa02000088
:020000040000fa
:04009c00fa02000064
:020000040000fa
:0401b800fa02000047
:020000040000fa
:0401bc00fa02000043
:020000040000fa
:0401c000fa0200003f
:020000040000fa
:0401c400fa0200003b
:020000040000fa
:0401c800fa02000037
:020000040000fa
:0401cc00fa02000033
:020000040000fa
:0401d000fa0200002f
:020000040000fa
:0401d400fa0200002b
:020000040000fa
:0401d800fa02000027
:020000040000fa
:0401dc00fa02000023
:020000040000fa
:0401e000fa0200001f
:020000040000fa
:0401e400fa0200001b
:020000040000fa
:0401e800fa02000017
:020000040000fa
:0401ec00fa02000013
:020000040000fa
:0401f000fa0200000f
:020000040000fa
:0401f400fa0200000b
:020000040000fa
:0401f800fa02000007
:020000040000fa
:0401fc00fa02000003
:020000040000fa
:04020000fa020000fe
:020000040000fa
:04020400fa020000fa
:020000040000fa
:04020800fa020000f6
:020000040000fa
:04020c00fa020000f2
:020000040000fa
:04021000fa020000ee
:020000040000fa
:04021400fa020000ea
:020000040000fa
:04021800fa020000e6
:020000040000fa
:04021c00fa020000e2
:020000040000fa
:04022000fa020000de
:020000040000fa
:04022400fa020000da
:020000040000fa
:04022800fa020000d6
:020000040000fa
:04022c00fa020000d2
:020000040000fa
:04023000fa020000ce
:020000040000fa
:04023400fa020000ca
:020000040000fa
:04023800fa020000c6
:020000040000fa
:04023c00fa020000c2
:020000040000fa
:04024000fa020000be
:020000040000fa
:04024400fa020000ba
:020000040000fa
:04024800fa020000b6
:020000040000fa
:04024c00fa020000b2
:020000040000fa
:04025000fa020000ae
:020000040000fa
:04025400fa020000aa
:020000040000fa
:04025800fa020000a6
:020000040000fa
:04025c00fa020000a2
:020000040000fa
:04026800fa02000096
:020000040000fa
:04006400fa0200009c
:020000040000fa
:04007c00fa02000084
:020000040000fa
:04008000fa02000080
:020000040000fa
:04008400fa0200007c
:020000040000fa
:0400b000fa02000050
:020000040000fa
:0400b400fa0200004c
:020000040000fa
:0400c400fa0200003c
:020000040000fa
:0400c800fa02000038
:020000040000fa
:0400cc00fa02000034
:020000040000fa
:0400d000fa02000030
:020000040000fa
:0400d400fa0200002c
:020000040000fa
:0400d800fa02000028
:020000040000fa
:0400dc00fa02000024
:020000040000fa
:0400e000fa02000020
:020000040000fa
:0400e400fa0200001c
:020000040000fa
:0400e800fa02000018
:020000040000fa
:0400f400fa0200000c
:020000040000fa
:0400f800fa02000008
:020000040000fa
:0400fc00fa02000004
:020000040000fa
:04010000fa020000ff
:020000040000fa
:04010400fa020000fb
:020000040000fa
:04010800fa020000f7
:020000040000fa
:04010c00fa020000f3
:020000040000fa
:04011400fa020000eb
:020000040000fa
:04011800fa020000e7
:020000040000fa
:04011c00fa020000e3
:020000040000fa
:04012000fa020000df
:020000040000fa
:04012400fa020000db
:020000040000fa
:04012800fa020000d7
:020000040000fa
:04013800fa020000c7
:020000040000fa
:04013c00fa020000c3
:020000040000fa
:04014000fa020000bf
:020000040000fa
:04014400fa020000bb
:020000040000fa
:04014800fa020000b7
:020000040000fa
:04014c00fa020000b3
:020000040000fa
:04015000fa020000af
:020000040000fa
:04015400fa020000ab
:020000040000fa
:04015800fa020000a7
:020000040000fa
:04016000fa0200009f
:020000040000fa
:04016400fa0200009b
:020000040000fa
:04016800fa02000097
:020000040000fa
:04016c00fa02000093
:020000040000fa
:04017000fa0200008f
:020000040000fa
:04017400fa0200008b
:020000040000fa
:04017800fa02000087
:020000040000fa
:04017c00fa02000083
:020000040000fa
:04018000fa0200007f
:020000040000fa
:04018400fa0200007b
:020000040000fa
:04018800fa02000077
:020000040000fa
:04018c00fa02000073
:020000040000fa
:04019000fa0200006f
:020000040000fa
:04019400fa0200006b
:020000040000fa
:04019800fa02000067
:020000040000fa
:04019c00fa02000063
:020000040000fa
:0401a000fa0200005f
:020000040000fa
:0401a400fa0200005b
:020000040000fa
:0401a800fa02000057
:020000040000fa
:0401ac00fa02000053
:020000040000fa
:0401b000fa0200004f
:020000040000fa
:0401b400fa0200004b
:020000040000fa
:04026400fa0200009a
:020000040000fa
:04006c00fa02000094
:020000040000fa
:0400f000fa02000010
:020000040000fa
:04001800fa020000e8
:020000040000fa
:04003000fa020000d0
:020000040000fa
:04004000fa020000c0
:020000040000fa
:04008c00fa02000074
:020000040000fa
:04009000fa02000070
:020000040000fa
:04000800fa020000f8
:020000040000fa
:04027400fa0200008a
:020000040000fa
:04027800fa02000086
:020000040000fa
:04027c00fa02000082
:020000040000fa
:04028000fa0200007e
:020000040000fa
:04026c00fa02000092
:020000040000fa
:04027000fa0200008e
:020000040000fa
:04011000fa020000ef
:020000040000fa
:04002400fa020000dc
:020000040000fa
:04006800fa02000098
:020000040000fa
:0400ec00fa02000014
:020000040000fa
:04004c00fa020000b4
:020000040000fa
:04005000fa020000b0
:020000040000fa
:0400a800fa02000058
:020000040000fa
:0400ac00fa02000054
:020000040000fa
:04002000fa020000e0
:020000040000fa
:04001400fa020000ec
:020000040000fa
:04003400fa020000cc
:020000040000fa
:04004400fa020000bc
:020000040000fa
:04004800fa020000b8
:020000040000fa
:04009400fa0200006c
:020000040000fa
:04009800fa02000068
:020000040000fa
:04012c00fa020000d3
:020000040000fa
:04005400fa020000ac
:020000040000fa
:04005800fa020000a8
:020000040000fa
:04013000fa020000cf
:020000040000fa
:0400a000fa02000060
:020000040000fa
:0400a400fa0200005c
:020000040000fa
:080000000002040000000000f2
:020000040000fa
:100400000f0021000eff21000e01880000000000f7
:10041000000020000000e000020032000001200087
:100420002002880014000700740007000000e000ac
:1004300003003a0000002000010020000200370005
:100440000000200001002000810f70000100320038
:100450000f000700000020000000e0000200320052
:100460000000020000000000100602000000000072
:100470000040da000000fe00200020000000e00044
:1004800002003200100020009001880000000600e9
:10049000a1028800800478000000eb001f003700f4
:1004a000e284440054a0b4009905ba00e2844400f8
:1004b00054a0b4009906ba00e284440054a0b400e9
:1004c0000006eb00476fde00fd07b200ae018800ba
:1004d000636ce10003003a000ad801000000eb0061
:1004e0000e003700606ce10008003a00004deb00a0
:1004f0000a05e800020039003420ec000af0a000f0
:100500008b05e900f9ff3e00040037006168e10057
:10051000010032000086eb000b00070019c7ba008b
:100520000e04e0001905ba0003003a000a00e000da
:10053000dbff3a0000000600fe07b200ae028800b2
:100540008a047800f5ff37000cd0a300e20f4d00bd
:100550001c00390089027800354dba000a05e80010
:10056000020039003420ec000af0a0008b05e900fd
:100570000f003200254dba000a05e80002003900dc
:100580003420ec000af0a0008b05e90008003200de
:100590000c00e0000600320015cdba000a05e800a4
:1005a000020039003420ec000af0a0008b05e900bd
:1005b0008984e80054a0b4000b00e000e2ff3a0098
:1005c000000006009902ba00055d78008b05e9007d
:1005d000f7ff3200c82ade00055d78008b05e900d0
:1005e000f3ff32000c00e000f1ff320019ddba0029
:1005f000eeff37000040da000000fe0000000500ba
:1006000003f0a200889fbe008a9fbe008c1f780066
:10061000b7000700be0033006450e1004f00320015
:100620006420e1005200320003826c0007003b00ae
:100630000905d0000306d000820f54000c065d00af
:1006400002003900020032008901780003067800b8
:100650008582550004003d000003fd008103fd007c
:100660008502ea008b854200840f720002003b0085
:1006700060001000e08018006011b8000005eb0079
:100680007a28e1000a00390006007800c75ddd0025
:10069000f707b200878075002d0037008281710056
:1006a0000a017800610560008180d1000080d300dc
:1006b0008502e900f9ff3b000604400087844800fa
:1006c00002003b0060041400e0841c000988a300c1
:1006d000070032008a81710082817100610164002b
:1006e0008904d1000884d3008b05e8001700370087
:1006f0000978a30013003a000b00e0001300340057
:100700008b05e9000804440089844c000a44740005
:100710000978a3000d003a000b00e0000700340048
:100720008b05e9000804440089844c0001003a006c
:100730000b0020000978a300f7ff32000001eb0056
:1007400002003700828171000a0178002d00070045
:100750000cf0a70001f0a000760037006420e10053
:1007600002003a00838f6c00760033000801be005f
:100770000200be006f0037000001be004700070006
:100780000470a70003f0a1006509b1001600320053
:100790000d0035006828e10006003500f0ff2f004d
:1007a000f1ff27000300e00013003b0001002800d8
:1007b0000000050000004000818048008502e9003b
:1007c000fcff3a0008003700f88f420002003c00ae
:1007d0008000eb00000005008100d1000080d30004
:1007e0008502e800fcff3a000300e00002003b0045
:1007f00060001000e0801800000006006011b800e2
:100800008700370081002000618055000b003d000b
:100810000b00200061fe2f000100e1001d003400ec
:1008200082817100610164008904d1000884d300d1
:100830000000e800faff3a00710020006100640047
:1008400003007000020060000900320061044400ef
:10085000e0844c000988a500050032008b05e80003
:100860006808e10002003a008904d1000884d3003e
:10087000f20f20000258e10005003d00c75ddd00d9
:10088000f907b200898075000800780000000600b2
:100890000bf827008b00780000000500c70ade0077
:1008a000f107b200f50fb20008003200e1cf4200bc
:1008b000020032000170a00024000500810f7000ca
:1008c000010032000408050044000500810f70009b
:1008d00002003a00140005008502e9000000400013
:1008e00081c04800fcff3b000170a000240005000f
:1008f0000004be00e9ff07000003be000405be00bf
:100900000200be00e5ff0700844f750000000600ee
:100910000200be006450e100050036006420e100e2
:10092000020036000968a30001003a000800be007a
:100930000160a0004f0678004f05be004f04be00c6
:1009400000000600f0ff2f00f1ff2700f9ff37003d
:10095000889fbe008a9fbe008c1f7800e4ff0700be
:10096000ebff330003866c006450e100240032008a
:100970006420e100270032006150e10022003200d3
:100980006120e100210032008b854200eb07b100bd
:100990000134b800003ab8000804420089844a00d3
:1009a000013ab8000030b8008880400009014a00d0
:1009b000040033000000400081804800020149002b
:1009c0008b05e900c909dd008301700001003200d8
:1009d00013002000c814de004814dd004709de00c3
:1009e0001200b200c808de000884700085ff07000e
:1009f00001f0a1000cf0a70001f0a000cdff37002e
:100a00006120e100cfff32000801be000200be00fd
:100a1000f7ff37006150e100fcff3a00c9ff3700e3
:100a2000889fbe008a9fbe00008270000402710091
:100a300004827100260032000004be000200be00e5
:100a40006011b8006b092000950220000182cf00e0
:100a50000a0039000541b1000082cf0007003900cb
:100a60000541b1000982cf00040039000541b10001
:100a70000882cf00010039000541b1000542520053
:100a8000120032000a003b008281710061016400a3
:100a90008100d1000080d3008984d3000884d30072
:100aa0008b05e8000442e800f7ff3a000700370032
:100ab0000804440089844c000000480081804800fc
:100ac0008b05e9000442e900f9ff3a004dff0700f9
:0c0ad0004f05be004f04be0000000600f1
:020000040000fa
:04aff400ffff00005b
:020000040000fa
:04aff00078ff0000e6
:020000040000fa
:04afe8007fff0000e7
:020000040000fa
:04afe000cfff00009f
:020000040000fa
:100adc000000fa0040002000001988002223ef00db
:100aec00f0002000201988003223ef005000200075
:100afc00401988002623ef002e23ef003023ef004f
:100b0c0011198000f0ff210000806000101988008e
:100b1c0025e3a80001198000f0cf2f0000806000b1
:100b2c000019880021e3a8000080fa0000000600ec
:100b3c000200fa002023a900000000000019800028
:100b4c00610060000000e000fcff32002003a900ff
:100b5c00001880008000eb0025ff0700626626006d
:100b6c006302240077ff07000001be0000002c0088
:100b7c00f14f24009ffe0700fcfe0700000f7800d9
:100b8c001e0078000000e000020034001e00780017
:100b9c00010037000000eb000080fa0000000600a6
:100bac000400fa009070800080007800000820009b
:100bbc000080600010079800000000009170800019
:100bcc0000082000808060001e009000808f500084
:100bdc00faff320040c6b300004f78000100370026
:100bec001e4fe9001e4078000004e000fcff3c00b2
:100bfc0000000000917080000008200080806000e0
:100c0c001e009000808f5000faff3a000080fa001e
:100c1c00000006000808fa000e2eef0080002000ed
:100c2c00f0708800002eef000080eb0080708800d0
:100c3c001c2eef0070f72f00d0708800a4ff070067
:100c4c000040eb00504798004000200020708800c6
:100c5c00c01220003007980004003700d0ff0700b6
:100c6c003e0090000000e900300798003e00900024
:100c7c000000e000f9ff3c0010002000207088000c
:100c8c00c01220003007980004003700c4ff070092
:100c9c003e0090000000e900300798003e009000f4
:100cac000000e000f9ff3c002000200020708800cc
:100cbc00c01220003007980004003700b8ff07006e
:100ccc003e0090000000e900300798003e009000c4
:100cdc000000e000f9ff3c00042eef00690f470014
:100cec0093ff070010079800010037000000000078
:100cfc00abff0700907080000040780067406000f8
:100d0c00004f98001e0090000000e0002f00320001
:100d1c005e4090000004e0001e0032000040eb003a
:100d2c00504798008e489000400020000008dd00dd
:100d3c00004f98001e007800904078000e489000fc
:100d4c0080c070001e007800014878001e0fe8007b
:100d5c009e007800690047000080500080007800f9
:100d6c001e009000808f500003003600690f470072
:100d7c006fff0700100798004e4090000080fb00aa
:100d8c000080ea004480de0067006000207088006c
:100d9c00d7ff370010c0b300504798001e007800f2
:100dac0090407800414798001e0078008e489000d3
:100dbc00014878004e4090000080fb000080ea0063
:100dcc006700600020708800c9ff37003e0090006b
:100ddc000000e800300798000e4890000080fb00ef
:100dec000080ea0020708800be00900000e2240021
:100dfc00808f5000bdff34004dff07001007980096
:0c0e0c000000eb0030079800b9ff370031
:00000001FF
